:020000001F29B6
:08000800FF0003088301FE0064
:100010000A08FD0000308A003F29A101A117B400A1
:10002000FE30892034088928A0112408031D1B28CC
:10003000A0150A30A4003808A8003708A700360821
:10004000A6003508A500A301B001AF01AE010A303A
:10005000AD00A120A30A23082402031D24282D0893
:10006000031DA011A01D3628240B39282D08303E71
:100070008920A40B1B281B29B200861106118316A8
:10008000861106110F30860583123208A0186628E3
:100090003E30A60080308D203330B1007A201330FE
:1000A000A60088308D207A2064308C207A2064303D
:1000B0008C202230B1007A20283065200C30652059
:1000C00006306520A014320866282014B100201CD8
:1000D00074280611033C031C792879200730A600F8
:1000E000D0308D20031408002014FE3C031987280B
:1000F0000615201C201086150F3086053108F039B2
:1001000086048611B10E20187A2832308C203208ED
:100110001B29A11B3C280800A601E83EA500A60952
:10012000FC30031C9628A50703189328A507000098
:10013000A60F932825189C28A51CA0280000A028FD
:100140000800280830068039B200A81FB228A50987
:10015000A609A709A809A50A0319A60A0319A70A47
:100160000319A80AB01FBF28AD09AE09AF09B0092D
:10017000AD0A0319AE0A0319AF0A0319B00AA9019F
:10018000AA01AB01AC01B901BA01BB01BC01300845
:100190002F042E042D040319FD282030B100031074
:1001A000A50DA60DA70DA80DB90DBA0DBB0DBC0D63
:1001B00030083C02031DE6282F083B02031DE628F9
:1001C0002E083A02031DE6282D083902031CF728E1
:1001D0002D08B9022E08031C2E0FBA022F08031C8B
:1001E0002F0FBB023008031C300FBC020314A90DF3
:1001F000AA0DAB0DAC0DB10BCF28B21F0A29A9096E
:10020000AA09AB09AC09A90A0319AA0A0319AB0A7E
:100210000319AC0A3908AD003A08AE003B08AF003C
:100220003C08B0002908A5002A08A6002B08A70052
:100230002C08A8001B298313831203130800A001B4
:1002400083168117FF309C009F01013086008312C6
:1002500086018530831681006430831281008B16FD
:10026000E7308E00FF308F0020309000101483168E
:100270000C140B178B1783128A110A126C298A111E
:100280000A120B1D52290130C10703010318013066
:10029000C207030103180130C3070301031801302B
:1002A000C4070B118A110A120C1C65290130BD0705
:1002B000030103180130BE07030103180130BF0713
:1002C000030103180130C0070C107D088A007E0866
:1002D0008300FF0E7F0E09008030A1008A010D20EF
:1002E000A4014008B8003F08B7003E08B6003D082A
:1002F000B5008A0114208030A100C0308A010D2091
:10030000A4014408B8004308B7004208B6004108F9
:0E031000B5008A0114208A016C298A018D290A
:02400E00323F3F
:00000001FF
